:020000040800F2
:1000000000070020F504000899300008513000086E
:10001000793000085130000871300008F7040008FA
:10002000F7040008F7040008F70400087940000806
:10003000F7040008F7040008F7040008F7040008B4
:10004000F7040008F7040008F7040008F7040008A4
:10005000F7040008F7040008C9530008F15300082A
:10006000195400084154000869540008F7040008B6
:10007000F7040008F7040008F7040008F704000874
:10008000F7040008F7040008F7040008F704000864
:10009000F7040008013000081530000891540008EA
:1000A000F7040008F7040008F7040008F704000844
:1000B00079550008F7040008F7040008F704000861
:1000C000F7040008F7040008F7040008F704000824
:1000D000F7040008F704000865550008F704000855
:1000E000F5540008F7040008F7040008F7040008B6
:1000F000F7040008F7040008F7040008F7040008F4
:10010000F7040008F7040008F7040008F7040008E3
:10011000F7040008F7040008F7040008F7040008D3
:10012000F7040008F7040008F7040008F7040008C3
:10013000F7040008F7040008F7040008F7040008B3
:10014000F7040008F7040008F7040008F7040008A3
:10015000F7040008F7040008F7040008F704000893
:10016000F7040008F7040008F7040008F704000883
:10017000F7040008F7040008F7040008F704000873
:10018000F7040008F7040008F7040008F704000863
:10019000F7040008F7040008293000083D30000883
:1001A000F7040008F7040008F7040008F704000843
:1001B000F7040008F7040008F7040008F704000833
:1001C000F7040008F7040008F7040008F704000823
:1001D000F7040008F7040008F7040008F704000813
:1001E00045180008000000000000000000000000AA
:1001F00053B94AB9002908BF00281CBF4FF0FF318E
:100200004FF0FF3000F074B9ADF1080C6DE904CE89
:1002100000F006F8DDF804E0DDE9022304B07047E1
:100220002DE9F047089D04468E46002B4DD18A42A9
:10023000944669D9B2FA82F252B101FA02F3C2F1DC
:10024000200120FA01F10CFA02FC41EA030E94406D
:100250004FEA1C48210CBEFBF8F61FFA8CF708FB8E
:1002600016E341EA034306FB07F199420AD91CEB66
:10027000030306F1FF3080F01F81994240F21C8198
:10028000023E63445B1AA4B2B3FBF8F008FB1033E0
:1002900044EA034400FB07F7A7420AD91CEB040415
:1002A00000F1FF3380F00A81A74240F207816444E5
:1002B000023840EA0640E41B00261DB1D44000236A
:1002C000C5E900433146BDE8F0878B4209D9002DCE
:1002D00000F0EF800026C5E9000130463146BDE858
:1002E000F087B3FA83F6002E4AD18B4202D38242C2
:1002F00000F2F980841A61EB030301209E46002D71
:10030000E0D0C5E9004EDDE702B9FFDEB2FA82F2C5
:10031000002A40F09280A1EB0C014FEA1C471FFA23
:100320008CFE0126200CB1FBF7F307FB131140EA0A
:1003300001410EFB03F0884208D91CEB010103F1D7
:10034000FF3802D2884200F2CB804346091AA4B299
:10035000B1FBF7F007FB101144EA01440EFB00FE6D
:10036000A64508D91CEB040400F1FF3102D2A645D2
:1003700000F2BB800846A4EB0E0440EA03409CE771
:10038000C6F12007B34022FA07FC4CEA030C20FA1E
:1003900007F401FA06F31C43F9404FEA1C4900FA3E
:1003A00006F3B1FBF9F8200C1FFA8CFE09FB1811BB
:1003B00040EA014108FB0EF0884202FA06F20BD92E
:1003C0001CEB010108F1FF3A80F08880884240F27E
:1003D0008580A8F102086144091AA4B2B1FBF9F0C2
:1003E00009FB101144EA014100FB0EFE8E4508D9BD
:1003F0001CEB010100F1FF346CD28E456AD9023842
:10040000614440EA0840A0FB0294A1EB0E01A14226
:10041000C846A64656D353D05DB1B3EB080261EB94
:100420000E0101FA07F722FA06F3F1401F43C5E96E
:10043000007100263146BDE8F087C2F12003D840A4
:100440000CFA02FC21FA03F3914001434FEA1C47E6
:100450001FFA8CFEB3FBF7F007FB10360B0C43EAD8
:10046000064300FB0EF69E4204FA02F408D91CEB88
:10047000030300F1FF382FD29E422DD90238634486
:100480009B1B89B2B3FBF7F607FB163341EA034126
:1004900006FB0EF38B4208D91CEB010106F1FF3875
:1004A00016D28B4214D9023E6144C91A46EA00466C
:1004B00038E72E46284605E70646E3E61846F8E6FE
:1004C0004B45A9D2B9EB020864EB0C0E0138A3E747
:1004D0004646EAE7204694E74046D1E7D0467BE728
:1004E000023B614432E7304609E76444023842E7A0
:1004F000704700BF02E000F000F8FEE772B6374830
:1005000080F30888364880F3098836483649086001
:1005100040F20000CCF200004EF63471CEF2000141
:100520000860BFF34F8FBFF36F8F40F20000C0F23F
:10053000F0004EF68851CEF200010860BFF34F8FF5
:10054000BFF36F8F4FF00000E1EE100A4EF63C71E2
:10055000CEF200010860062080F31488BFF36F8F8D
:1005600004F062FD04F0F4FD4FF055301F491B4AC2
:1005700091423CBF41F8040BFAE71D49184A9142E9
:100580003CBF41F8040BFAE71A491B4A1B4B9A423D
:100590003EBF51F8040B42F8040BF8E7002018495D
:1005A000184A91423CBF41F8040BFAE704F040FDC1
:1005B00004F014FE144C154DAC4203DA54F8041B3D
:1005C0008847F9E700F042F8114C124DAC4203DACB
:1005D00054F8041B8847F9E704F028BD0007002001
:1005E000002300200000000808ED00E000010020CA
:1005F0000007002090580008002300208C230020D2
:100600009023002078690020E0010008E401000840
:10061000E4010008E40100082DE9F04F2DED108AF7
:10062000C1F80CD0C3689D46BDEC108ABDE8F08FC0
:10063000002383F311882846A047002004F082F9A4
:10064000FEE704F0E5F800DFFEE70000F8B501F092
:100650000FF904F08BFC074604F0DCFC0546B8BB40
:10066000204B9F4234D001339F4234D01E4B27F0A1
:10067000FF029A4232D1F8B200F028FF2E4642F231
:10068000107400F029FF08B10024264601F07CFC1C
:1006900020B1032000F07CF80024264635B1134B2E
:1006A0009F4203D004F0AEFC00242646002004F054
:1006B00067FC0EB100F082F801F04CFA00F03EFF4A
:1006C00001F034F9204600F0D1F800F077F8F9E7AE
:1006D0002E460024D5E704460126D2E7064640F61A
:1006E000C414CEE7010007B0000008B0263A09B0F4
:1006F00008B501F0E7F8A0F120035842584108BDC1
:1007000007B541F21203022101A8ADF8043001F04F
:10071000F7F803B05DF804FB38B5302383F3118894
:10072000174803680BB104F0CBF9164A14480023AC
:100730004FF47A7104F0BAF9002383F31188124C54
:10074000236813B12368013B2360636813B16368B6
:10075000013B63600D4D2B7833B963687BB9022090
:1007600001F086F9322363602B78032B07D163688D
:100770002BB9022001F07CF94FF47A73636038BD25
:100780009023002019070008B0240020A82300208F
:10079000084B187003280CD8DFE800F008050208A1
:1007A000022001F05BB9022001F04EB9024B002299
:1007B0005A607047A8230020B024002010B501F033
:1007C000E3FB30B1234B03221A70234B00225A6003
:1007D00010BD224B224A1C4619680131F8D004335F
:1007E0009342F9D16268A242F2D31E4B9B6803F197
:1007F000006303F510439A42EAD204F0D5FB04F0FB
:10080000E7FB002001F0ACF80220FFF7C1FF164B18
:100810009A6D00229A65996F9A67996FD96DDA651A
:10082000D96FDA67D96F196E1A66D3F88010C3F8DA
:100830008020D3F8803072B64FF0E0233021C3F827
:10084000084DD4E9003281F311889D4683F308886E
:100850001047BDE7A8230020B02400200090000826
:100860002090000800230020001002402DE9F04FE6
:1008700093B0AC4B00902022FF210AA89D6801F0A4
:1008800013F9A94A1378A3B9A8480121036011708C
:10089000302383F3118803680BB104F011F9A44AE3
:1008A000A24800234FF47A7104F000F9002383F387
:1008B0001188009B13B19F4B009A1A609E4A009CBE
:1008C0001378032B1EBF002313709A4A4FF0000ABF
:1008D00018BF5360D3465646D146012001F0BEF8FA
:1008E00024B1944B1B68002B00F01582002000F00F
:1008F000E9FF0390039B002B01DA00F073FE039BDA
:10090000002BEDDB012001F09FF8039B213B162B10
:10091000E3D801A252F823F0750900089D090008E8
:10092000310A0008DB080008DB080008DB080008C3
:10093000BB0A00088B0C0008A50B0008070C000878
:100940002F0C0008550C0008DB080008670C000895
:10095000DB080008D90C0008150A0008DB080008AD
:100960001D0D000881090008150A0008DB080008B1
:10097000070C00080220FFF7BBFE002840F0F581BD
:10098000009B0221BAF1000F08BF1C4605A841F2E6
:100990001233ADF8143000F0B3FF9EE74FF47A70D5
:1009A00000F090FF071EEBDB0220FFF7A1FE0028FE
:1009B000E6D0013F052F00F2DA81DFE807F0030AF5
:1009C0000D10133605230593042105A800F098FFA8
:1009D00017E054480421F9E758480421F6E758483D
:1009E0000421F3E74FF01C08404600F0BBFF08F17C
:1009F00004080590042105A800F082FFB8F12C0F2F
:100A0000F2D1012000FA07F747EA0B0B5FFA8BFBE4
:100A10004FF0000901F094F826B10BF00B030B2BFB
:100A200008BF0024FFF76CFE57E746480421CDE7D6
:100A3000002EA5D00BF00B030B2BA1D10220FFF74A
:100A400057FE074600289BD0012000F089FF0220B6
:100A5000FFF79EFE00261FFA86F8404600F090FF42
:100A6000044690B10021404600F0A2FF0136002864
:100A7000F1D1BA46044641F21213022105A8ADF89D
:100A800014303E4600F03CFF27E70120FFF780FED0
:100A90002546244B9B68AB4207D9284600F062FFED
:100AA000013040F067810435F3E7234B00251D70CA
:100AB000204BBA465D603E46ACE7002E3FF460AF87
:100AC0000BF00B030B2B7FF45BAF0220FFF760FEF4
:100AD000322000F0F7FEB0F10008FFF651AF18F039
:100AE00003077FF44DAF0F4A926808EB050393426A
:100AF0003FF646AFB8F5807F3FF742AF124B019308
:100B0000B84523DD4FF47A7000F0DCFE0390039AC1
:100B1000002AFFF635AF019B039A03F8012B01373A
:100B2000EDE700BF00230020AC240020902300202C
:100B300019070008B0240020A82300200423002067
:100B4000082300200C230020AC230020C820FFF73E
:100B5000CFFD074600283FF413AF1F2D11D8C5F174
:100B6000200242450AAB25F0030028BF42468349D4
:100B70000192184400F086FF019A8048FF2100F09E
:100B800093FF4FEAA8037D490193C8F387022846E3
:100B900000F092FF064600283FF46DAF019B05EB85
:100BA000830537E70220FFF7A3FD00283FF4E8AEF6
:100BB00000F010FF00283FF4E3AE0027B846704B6A
:100BC0009B68BB4218D91F2F11D80A9B01330ED046
:100BD00027F0030312AA134453F8203C0593404620
:100BE000042205A901F0BAF904378046E7E7384640
:100BF00000F0B8FE0590F2E7CDF81480042105A8B6
:100C000000F07EFE06E70023642104A8049300F0B0
:100C10006DFE00287FF4B4AE0220FFF769FD0028C6
:100C20003FF4AEAE049800F0CBFE0590E6E700235B
:100C3000642104A8049300F059FE00287FF4A0AEBC
:100C40000220FFF755FD00283FF49AAE049800F00B
:100C5000B9FEEAE70220FFF74BFD00283FF490AE13
:100C600000F0C8FEE1E70220FFF742FD00283FF454
:100C700087AE05A9142000F0C3FE042107460490A6
:100C800004A800F03DFE3946B9E7322000F01AFE14
:100C9000071EFFF675AEBB077FF472AE384A926846
:100CA00007EB090393423FF66BAE0220FFF720FDEE
:100CB00000283FF465AE27F003074F44B9453FF4E1
:100CC000A9AE484600F04EFE0421059005A800F0AC
:100CD00017FE09F10409F1E74FF47A70FFF708FDF8
:100CE00000283FF44DAE00F075FE002844D00A9B6A
:100CF00001330BD008220AA9002000F0DDFE0028F5
:100D00003AD02022FF210AA800F0CEFEFFF7F8FC1F
:100D10001C4803F01DFE13B0BDE8F08F002E3FF419
:100D20002FAE0BF00B030B2B7FF42AAE00236421B4
:100D300005A8059300F0DAFD074600287FF420AEF1
:100D40000220FFF7D5FC804600283FF419AEFFF7DC
:100D5000D7FC41F2883003F0FBFD059800F006FF58
:100D6000464600F0EDFE3C46B7E5064652E64FF03B
:100D7000000905E6BA467EE637467CE6AC2300204D
:100D800000230020A0860100094A136849F2690087
:100D900099B21B0C00FB01331360064B186844F238
:100DA000506182B2000C01FB0200186080B27047F3
:100DB000142300201023002010B500211022044627
:100DC00000F072FE034B03CB206061601868A060E6
:100DD00010BD00BF9075FF1F2DE9F041ADF54E7DB0
:100DE0000DF134086CAC40F2751207460D460EA8A2
:100DF0000021C8F8001000F057FE4FF4C472002123
:100E0000204600F051FE02F04FF9274B4FF47A7262
:100E1000B0FBF2F0186093E80700022384E80700B3
:100E20000DF5E9702382FFF7C7FF41F604531F4910
:100E3000238406A804F03CFC1B2384F832310DF215
:100E4000E32206AB0DF1300C1E4603CE6645106062
:100E50005160334602F10802F6D13188B3789370BD
:100E6000118020464146012200F09AFE00230393A0
:100E7000AB7E029305F11903019380B20123CDE902
:100E800004800093E97E06A3D3E90023384602F0EC
:100E9000C9FC0DF54E7DBDE8F08100BFAFF30080C9
:100EA0009E6AC421818A46EEB8240020C0560008FC
:100EB0002DE9F0412C4C237ADAB080460D465BBB1D
:100EC00027A9284600F07CFF0746002842D19DF85C
:100ED0009D60C82E3ED801464FF4A662204600F021
:100EE000E3FD4FF48073C4F8F8314FF40073C4F895
:100EF0000C334FF44073C4F8203432460DF19E0198
:100F000004F1090000F0BEFD26449DF89C30777284
:100F100023720BB9EB7E23728122002106AC27A835
:100F200000F0C2FD0122214627A800F085FF002322
:100F30000393AB7E029305F1190380B2019328233A
:100F4000CDE904400093E97E05A3D3E900234046A0
:100F500002F068FC5AB0BDE8F08100BFAFF300803A
:100F600026417272DF25D7B7605E0020F0B5254EAE
:100F70004FF48A7505FB0065F1B096F8D83085F816
:100F8000DC300024D822214685F8E8403AA800F059
:100F90008BFD06F1090000F07FFDD5F8E4308DF8F7
:100FA000F000C2B206AF06F109010DF1F100CDE982
:100FB0003A3400F067FD394601223AA800F068FF94
:100FC00080B2CDE9047008230127CDE9023706F18C
:100FD000D803019330230093317A0B4807A3D3E958
:100FE000002302F01FFCA04206DD02F05DF8C5F808
:100FF000E000384671B0F0BD2046FBE778F6339F3D
:1010000093CACD8D605E0020D03400202DE9F04FD2
:10101000274FDFF8A880274E87B0384602F02EFC15
:10102000034600283DD00024CDE90344ADF8144028
:10103000027B8DF8142099684068029403AA03C2C9
:101040001B681D4D43F000430293A146A2462B6846
:10105000D3F810B002F02AF810EB080241F10003B7
:101060002846CDF800A002A9D84704F22C5440F637
:1010700058230028C8BF49F0010905F5A5559C4231
:1010800005F11005E3D1B9F1000F05D0384602F0A3
:10109000F9FB86F800A0C0E73378072B04D80133AA
:1010A000337007B0BDE8F08F014802F0EBFBF8E7C2
:1010B000D0340020956300200035002040420F000E
:1010C00070B50D4614461E4602F008FB50B9022EBC
:1010D00010D1012C0ED112A3D3E90023C5E90023BE
:1010E000012007E0282C10D005D8012C09D0052CB0
:1010F0000FD0002070BD302CFBD10BA3D3E900230F
:10110000ECE70BA3D3E90023E8E70BA3D3E9002323
:10111000E4E70BA3D3E90023E0E700BFAFF30080CF
:10112000401DA12026812A0B78F6339F93CACD8DCE
:101130009E6AC421818A46EE26417272DF25D7B7A6
:10114000F017304A39059E5638B505460E4C002139
:10115000013500F02DFCA4F82C55B4F82C0500F056
:101160000FFC78B1B4F82C0500F01AFC014648B920
:10117000B4F82C0500F01CFCB4F82C350133A4F8AD
:101180002C35EAE738BD00BF605E0020F8B50E4C94
:101190000E4F0226A4F5805343F8307C237E3BB9E2
:1011A00065692DB1284600F06DFF284604F036FA37
:1011B000204600F067FFA4F5A554012EA4F1100409
:1011C00000D1F8BD0126E5E7E059002028570008C6
:1011D0002DE9F04F8FB000AF05460C4602F07EFAC5
:1011E000002849D1237E022B1BD1E38A012B18D181
:1011F00001F05AFF0646FFF7C7FD03464FF4C870DB
:10120000DFF8C482B3FBF0F206F5167602FB10336A
:1012100016FA83F3C8F80030E37E33B9A34B0022FB
:101220001A703C37BD46BDE8F08F07F12401204617
:1012300000F084FD0028F4D107F11400FFF7BCFD95
:1012400097F8264007F11401224607F1270004F021
:10125000FDF90028E2D10F2C08D8944B1C70D8F867
:101260000030A3F51673C8F80030DAE797F82410B9
:10127000284602F02BFAD4E7E38A282B2BD010D88B
:10128000012B23D0052BCCD1BFF34F8F8849894B3D
:10129000CA6802F4E0621343CB60BFF34F8F00BF14
:1012A000FDE7302BBDD1844EE17E327A9142B8D138
:1012B000607E3146002291F8DC50854200F0A58026
:1012C0000132042A01F58A71F5D1AAE721462846A0
:1012D000FFF782FDA5E721462846FFF7E9FDA0E7D5
:1012E000B2F8EC507B6005F103094FEA99094FEA27
:1012F0008902D11DC908A8EBC1039D46EB46002118
:10130000584600F0D1FB04F1EE012A46314458461C
:1013100000F0B8FB7B6813B9012000F021FB96F8C0
:10132000D20000F02DFB044630B9307200F052FBC1
:10133000204600F015FBB1E0D6F8D4203AB996F873
:10134000D200B6F82C25824201D8FFF7FDFED6F870
:10135000D4202A44944208D296F8D200B6F82C251C
:101360000130824201D8FFF7EFFE70685FFA89F220
:10137000594600F0A1FB08B9C54679E0726896F8B5
:10138000D2002A447260D6F8D42005EB0209C6F8D0
:10139000D49000F0F5FA814509D396F8D220D6F81A
:1013A000D4000132001B86F8D220C6F8D400FF2DED
:1013B0000FD80024347200F00DFB204600F0D0FA64
:1013C00000F0E2FD3D4B188108B9FFF7F7F9C5467B
:1013D00027E7BB6896F8D9000AFB0362FB68D2F8DE
:1013E000E41082F8E83001F58061C2F8E030C2F81C
:1013F000E410FFF7BBFDFFF709FE96F8D920013294
:1014000002F0030286F8D920B6E74FF48A7A0AFB85
:1014100002F505F1EA013144204600F065FDF8606F
:1014200000287FF4FEAE3544012285F8E82001F063
:101430003BFED5F8E020D6ED007ADFED216A801A78
:10144000192838BF192040F6B832904228BF1046FC
:10145000B8EE677A07EE900AF8EEE77A67EEA67ABA
:10146000DFED186AE7EE267AFCEEE77AC6ED007A41
:1014700096F8D930BB60BA6873680AFB02F4321977
:1014800092F8E81059B1D2F8E4108B42E8463FF4E4
:1014900027AF002182F8E810C2F8E010C546736853
:1014A000064A9B0A01331381BBE600BFC934002002
:1014B00000ED00E00400FA05605E0020B824002082
:1014C000CDCCCC3D6666663FCC340020014B187015
:1014D000704700BFC424002038B54FF00054134BB0
:1014E00022689A4220D1124B627D12481A70237DE5
:1014F00003724FF48073C0F8F8314FF40073C0F8F2
:101500000C3300254FF44073C0F820340A49C0F86A
:10151000E450C922093000F0B5FAE02229462046FD
:1015200000F0C2FA012038BD0020FCE79AAD44C5A6
:10153000C4240020605E00201600002037B500F0B3
:1015400023FD1F4C1F4D2049288102236B71236806
:10155000204604F580545B6801229847D4F8B034E3
:1015600019495B68012204F59660984700230193AE
:10157000164B174900931748174B4FF4805202F04F
:101580007DF8164B197811B1124802F09FF801F05E
:101590008BFD0446FFF7F8FB4FF4C873B0FBF3F282
:1015A00002FB130304F5167010FA83F00C4B18605D
:1015B00003F030FD08B10F232B8103B030BD00BF15
:1015C00000350020B824002040420F00C110000860
:1015D000C8240020D0340020D1110008C4240020E9
:1015E000CC3400202DE9F04F2DED028B002593B077
:1015F0000DF12C089FED838BDFF84492FFF706FD79
:101600000A95ADF834500B95C8F804500026834C69
:10161000DFF80CB2374601238DF81C3023688DF8B3
:101620001D508DED008B0DF11D02D3F808A007A908
:1016300000232046D0479DF81CA0BAF1000F24D00B
:10164000D9F8143083F48063C9F8143010220021D3
:101650000EA800F029FA236808AA5F690AA90DF10B
:101660001E032046B84798E803000FAB83E8030049
:101670009DF834308DF844300A9B0E930EA9DDE9B5
:101680000823584602F0DCFA574606F22C5640F67C
:10169000582304F5A5549E4204F11004BBD1002F39
:1016A000B4D15F4802F01AF800283FD15D4E01F036
:1016B000FBFC3368984239D301F0F6FC0446FFF78F
:1016C00063FB4FF4C873B0FBF3F202FB130304F5A2
:1016D000167010FA83F03060534E8DF8287037780A
:1016E00017B901238DF82830C7F11004E4B20EA811
:1016F000FFF762FB062C28BF06240EAB2246D91941
:101700000DF1290000F0BEF90AAB039318230293F0
:101710000134464B0193E4B2012300934048049402
:101720003AA3D3E9002302F01FF8357001F0BCFCA6
:101730003F4A404C1368C31AB3F57A7F2FD3106029
:1017400001F0B4FC02460B46354802F0A5F83448D7
:1017500001F0C4FF18B3237A374E002B14BF0323C4
:101760000223737101F0A0FC0EAF4FF47A730122D3
:10177000B0FBF3F039463060304600F0B7FA18237A
:1017800002932E4B019380B240F25513CDE90370C2
:10179000009323481FA3D3E9002301F0E5FF237A38
:1017A00093B101F081FC002607464FF48A7894F843
:1017B000D900304400F0030008FB004393F8E82010
:1017C00072B10136042EF2D1C82003F0C1F8237A99
:1017D000002B7FF40DAF13B0BDEC028BBDE8F08F92
:1017E000D3F8E02042B12368FA2B38BFFA23BA1AA3
:1017F0000533B2EB430FE4D3FFF7B8FB0028E0D189
:10180000E2E700BF0000000000000000401DA12032
:1018100026812A0BF1C6A7C1D068080F0035002029
:10182000D0340020CC340020C9340020C83400203B
:1018300090630020605E0020B824002094630020A4
:101840000008004808B5064800F052FF054800F0BF
:101850004FFFBDE80840044A0449002003F0D8BE09
:1018600000350020B0490020EC6300208D110008F5
:101870007047000070B5104B1B780133DBB2012BB1
:101880000C4612D80D4B1D6829684FF47A730E6A06
:10189000A2FB0332014622462846B047844204D1C7
:1018A000074B00221A70012070BD4FF4FA7003F04C
:1018B0004FF80020F8E700BF182300201C23002069
:1018C000DC63002007B50023024601210DF107006B
:1018D0008DF80730FFF7CEFF20B19DF8070003B069
:1018E0005DF804FB4FF0FF30F9E700000A4608B549
:1018F0000421FFF7BFFF80F00100C0B2404208BDE5
:1019000030B4074B0A461978064B53F82140236838
:10191000DD69054B0146AC46204630BC604700BF40
:10192000DC6300201C230020A086010070B503F0BA
:10193000B7F9094E094D3080002428683388834266
:1019400008D903F0A9F92B6804440133B4F5104F0A
:101950002B60F2D370BD00BFDE63002098630020CF
:1019600003F052BA00F1006000F5104000687047C3
:1019700000F10060920000F5104003F0CFB90000C4
:10198000054B1A68054B1B889B1A834202D91044E9
:1019900003F082B90020704798630020DE630020C6
:1019A000024B1B68184403F07FB900BF9863002006
:1019B000024B1B68184403F089B900BF98630020EC
:1019C0000020704700F10050A0F51040D0F89005BD
:1019D00070470000064991F8243033B10023086AAB
:1019E00081F824300822FFF7C3BF0120704700BFF1
:1019F0009C630020014B1868704700BF002004E082
:101A000030B50F4B0F4C1B682288C3F30B03013812
:101A1000934208440BD164680A46013C8242134653
:101A20000BD214F9015F2DB102F8015BF6E7814298
:101A30000B4602D22C2203F8012B581A30BD00BFEE
:101A4000002004E020230020022802BF024B4FF0B8
:101A500080629A61704700BF00080048022802BFF8
:101A6000024B4FF480629A61704700BF0008004843
:101A7000022801BF024A536983F4806353617047AF
:101A80000008004810B50023934203D0CC5CC45436
:101A90000133F9E710BD000003460246D01A12F9DF
:101AA000011B0029FAD1704702440346934202D039
:101AB00003F8011BFAE770472DE9F8431F4D144660
:101AC00095F824200746884652BBDFF870909CB3F7
:101AD00095F824302BB92022FF2148462F62FFF7CA
:101AE000E3FF95F82400C0F10802A24228BF224675
:101AF000D6B24146920005EB8000FFF7C3FF95F890
:101B00002430A41B1E44F6B2082E17449044E4B2BD
:101B100085F82460DBD1FFF75DFF0028D7D108E00E
:101B20002B6A03EB82038342CFD0FFF753FF0028D9
:101B3000CBD10020BDE8F8830120FBE79C630020A7
:101B4000024B1A78024B1A70704700BFDC6300200A
:101B50001823002003494FF461430B60024B1868BF
:101B600002F0BCBDC46300201C230020094B10B54B
:101B70001822044600211846FFF796FF064A074B35
:101B8000127804600146BDE8104053F8220002F0CC
:101B9000A5BD00BFC4630020DC6300201C2300201F
:101BA0002DE9F0470D46044600219046284640F2B4
:101BB0007912FFF779FF234620220021284601F001
:101BC000E1FF231D02222021284601F0DBFF631DD7
:101BD00003222221284601F0D5FFA31D032225213F
:101BE000284601F0CFFF04F10803102228212846DF
:101BF00001F0C8FF04F1100308223821284601F043
:101C0000C1FF04F1110308224021284601F0BAFF68
:101C100004F1120308224821284601F0B3FF04F121
:101C2000140320225021284601F0ACFF04F11803D0
:101C300040227021284601F0A5FF04F1200308226C
:101C4000B021284601F09EFF04F121030822B821AB
:101C5000284601F097FF04F12207C0263B46314693
:101C600008222846083601F08DFFB6F5A07F07F15F
:101C70000107F3D104F1320308223146284601F06E
:101C800081FF002704F1330A94F832304FEAC70984
:101C90009F4209F5A47615D3B8F1000F08D131465B
:101CA00004F599730722284601F06CFF09F24F16DC
:101CB000274694F832213B1B93420CD3F01DC008F9
:101CC000BDE8F0870AEB070308223146284601F0F9
:101CD00059FF0137D8E707F2331331460822284667
:101CE00001F050FF08360137E3E7000013B5044662
:101CF0000846002101602346C0F80310202201900D
:101D000001F040FF0198231D0222202101F03AFF3B
:101D10000198631D0322222101F034FF0198A31DC5
:101D20000322252101F02EFF019804F1080310225F
:101D3000282101F027FF072002B010BDF7B50023CE
:101D4000047F00910E4607221946054601F0DEFD8C
:101D5000731C0093012200230721284601F0D6FDC1
:101D6000C4B9B31C0093052223460821284601F07C
:101D7000CDFD0D243746B278BB1B934211D32B7F88
:101D8000A88A0734E408BBB9844294BF002001202C
:101D900003B0F0BDAB8ADB00083BDB08B37008245E
:101DA000E8E7FB1C0093214600230822284601F0A7
:101DB000ADFD08340137DEE7201A18BF0120E7E740
:101DC000F7B50023047F00910E4608221946054608
:101DD00001F09CFD731CC4B90822009311462346F0
:101DE000284601F093FD1024012372785F1C013B0B
:101DF000934211D32B7FA88A0734E408BBB98442ED
:101E000094BF0020012003B0F0BDAB8ADB00083B8B
:101E1000DB0873700824E7E7F319009321460023D9
:101E20000822284601F072FD08343B46DDE7201AFF
:101E300018BF0120E7E70000F8B50E460546144636
:101E4000002181223046FFF72FFE2B460822002179
:101E5000304601F097FE7CB96B1C07220821304602
:101E600001F090FE0F2401236A785F1C013B93422E
:101E700004D3E01DC008F8BD0824F4E7EB1921469F
:101E80000822304601F07EFE08343B46ECE70000B5
:101E9000F8B50E46054614460021CE223046FFF71F
:101EA00003FE2B4628220021304601F06BFE7CB950
:101EB00005F1080308222821304601F063FE302492
:101EC0002F462A7A7B1B934204D3E01DC008F8BD3D
:101ED0002824F5E707F1090321460822304601F0DE
:101EE00051FE08340137ECE7F7B5047F00910E4648
:101EF000012310220021054601F008FDC4B9B31CDE
:101F00000093092223461021284601F0FFFC1924E2
:101F100037467288BB1B9A4211D82B7FA88A073498
:101F2000E408BBB9844294BF0020012003B0F0BD97
:101F3000AB8ADB00103BDB0873801024E8E73B1D15
:101F40000093214600230822284601F0DFFC0834D4
:101F50000137DEE7201A18BF0120E7E730B5094D49
:101F60000A4491420DD011F8013B5840082340F338
:101F70000004013B2C4013F0FF0384EA5000F6D12B
:101F8000EFE730BD2083B8EDF7B5384A10685168E7
:101F90006B4603C36A4636493648082303F066FB9E
:101FA0000446002833D10A25334A106851686B462D
:101FB00003C36A4631492F48082303F057FB044600
:101FC000002849D00369B3F5EE2F45D8B0F8661064
:101FD00040F21D4291423FD1294A024402F15C0184
:101FE0008B4239D35C3B234900209E1AFFF7B6FF92
:101FF0003246074604F164010020FFF7AFFFA368F3
:102000009F4229D1E368984208BF002524E0036974
:10201000B3F5EE2F27D8418B40F21D42914220D1DB
:10202000174A024402F110018B4218D3103B1149A8
:1020300000209D1AFFF792FF2A46064604F1180178
:102040000020FFF78BFFA3689E4202D1E36898420D
:1020500001D00D25A8E70025284603B0F0BD1025C6
:10206000A2E70C25A0E70B259EE700BFE856000875
:10207000DC6F070000900008F1560008906F070021
:102080000870FFF710B5037C044613B9006803F02D
:10209000D5FA204610BD00000023BFF35B8FC3605C
:1020A000BFF35B8FBFF35B8F8360BFF35B8F7047C2
:1020B000BFF35B8F0068BFF35B8F704770B5054659
:1020C0000C30FFF7F5FF05F1080604463046FFF730
:1020D000EFFFA04206D930466D68FFF7E9FF2544BF
:1020E000281A70BD3046FFF7E3FF201AF9E7000019
:1020F00070B50546406898B105F10800FFF7D8FFB4
:1021000005F10C0604463046FFF7D2FF8442304604
:1021100094BF6D680025FFF7CBFF013C2C44201ACB
:1021200070BD000038B50C460546FFF7C7FFA0425A
:1021300010D305F10800FFF7BBFF04446868B4FB47
:10214000F0F100FB1144BFF35B8F0120AC60BFF3E3
:102150005B8F38BD0020FCE72DE9F04114460746AF
:102160000D46FFF7C5FF844228BF0446D4B1B846E8
:1021700058F80C6B4046FFF79BFF30442860404600
:102180007E68FFF795FF331A9C4203D86C600120EC
:10219000BDE8F0816B60A41B3B68AB602044E86045
:1021A0000220F5E72046F3E738B50C460546FFF771
:1021B0009FFFA04210D305F10C00FFF779FF044404
:1021C0006868B4FBF0F100FB1144BFF35B8F0120A2
:1021D000EC60BFF35B8F38BD0020FCE72DE9FF41C9
:1021E000884669460746FFF7B7FF6C4606B204EB20
:1021F000C6060025B44209D06268206808EB0501D4
:10220000FFF740FC636808341D44F3E7294638466D
:10221000FFF7CAFF284604B0BDE8F081F8B50546CF
:102220000C300F46FFF744FF05F108060446304620
:10223000FFF73EFFA042304688BF6C68FFF738FFCB
:10224000201A386020B130462C68FFF731FF204457
:10225000F8BD000073B5144606460D46FFF72EFF85
:10226000844228BF04460190DCB101A93046FFF743
:10227000D5FF019B33B93268C5E90233C5E90024B3
:1022800001200CE09C4238BF0194286001986860EE
:102290008442F5D93368AB60241AEC60022002B0A6
:1022A00070BD2046FBE700002DE9FF410F4669465F
:1022B000FFF7D0FF6C4600B204EBC0050026AC422D
:1022C00009D0D4F8048054F8081BB8194246FFF727
:1022D000D9FB4644F3E7304604B0BDE8F081000086
:1022E00038B50546FFF7E0FF044601462846FFF7EC
:1022F00019FF204638BD0000302383F3118862B6F1
:1023000070470000002383F3118862B67047000015
:10231000012070477047000010B41346026814682B
:102320000022A4465DF8044B6047000000F5805091
:1023300090F859047047000000F5805090F852045E
:102340007047000000F5805090F958047047000075
:102350005020704700F5805208B5FFF7CDFFD2F846
:102360009834D2F894041844D2F890341844D2F82F
:1023700078341844D2F888341844D2F88434184495
:10238000FFF7C0FF08BD000038B5C26A936923F0AB
:1023900001039361044600F087FE0546E36A9B69EA
:1023A000DB0706D500F080FE431BFA2BF6D9002090
:1023B00004E004F58054012084F8520438BD000084
:1023C0002DE9F04F0C4600F5805185B01F4691F87D
:1023D0005234BDF83890054690469BB1D1F874341C
:1023E0000133C1F8743423689A0006D4237B082B88
:1023F0000BD9627B0AB10F2B07D9D1F8783401339E
:10240000C1F878344FF0FF300FE0FFF775FFEB6A4B
:10241000D3F8C42012F4001A0AD0D1F87C34013366
:10242000C1F87C34FFF76EFF002005B0BDE8F08FE7
:10243000D3F8C46022686B6AC6F301464FF0480BBC
:10244000002A1BFB063BB4BF42F080429204CBF84B
:10245000002023685B0044BF42F00052CBF800200C
:10246000227B330643EA0243CBF80430607B7201DF
:1024700018B343F44013CBF80430D1F8A43401333B
:10248000C1F8A434AB1803F58353197B41F0200144
:102490001973207B039200F063FE039A03308010CF
:1024A0005FFA8AF383420AF1010A0DDA04EB830131
:1024B0000BEB830349689960F2E7AB1803F583538C
:1024C000197B60F34511E3E7EB6A0121B140C3F8E2
:1024D000CC10AB1803F58253C3E9048705EB461310
:1024E00003F582532146183304F10C0051F804CB54
:1024F00043F804CB8142F9D1098819802A4441F27A
:1025000068032846D65002F5805209F0030392F87A
:102510006C1043F0100321F01F010B4382F86C3064
:10252000FFF7F0FE4246CDF800903B46214600F012
:10253000DDFD012079E7000013B500F5805401911D
:10254000606CFFF7D5FD1F280AD90199606C202225
:10255000FFF744FEA0F120035842584102B010BDDD
:102560000020FBE708B500F58050FFF7C5FE406C82
:10257000FFF792FDBDE80840FFF7C4BE00220260ED
:10258000828142608260704710B500220023C0E95A
:1025900000230023044603810C30FFF7EFFF2046A1
:1025A00010BD00002DE9F047074688B007F58054BC
:1025B00068469A468846FFF79FFE9146FFF7E4FF7C
:1025C000606CFFF77BFD1F282CD9606C20226946C8
:1025D000FFF786FE202825D194F8523413B303ADBB
:1025E000444605AB2E4603CE9E42206061603546D0
:1025F00004F10804F6D130682060B388A380DDE9D7
:102600000023C9E90023BDF80830AAF80030FFF71D
:1026100079FE4A4653464146384608B0BDE8F04781
:1026200000F052BDFFF76EFE002008B0BDE8F08755
:102630002DE9F84F00230646C0E90133294B46F83F
:10264000303B00F5815405468846374610343846FD
:102650002037FFF799FFA742F9D105F580544FF4D1
:10266000805326630026C4E90D366764012305F50F
:10267000835705F5A359E66384F8403084F8483061
:10268000103709F110094FF0000A4FF0000B47E92D
:1026900008ABA7F11800FFF771FF203747F8286C47
:1026A0004F45F4D1B8F1010F84F85884A4F85A6466
:1026B000A4F85C64A4F85E6484F86064A4F86264BE
:1026C000A4F86464A4F8666484F8686402D90648CF
:1026D00000F0E4FC054B53F82830EB622846BDE8D7
:1026E000F88F00BF28570008FC560008185700084C
:1026F00010B5044B197804464A1C1A70FFF798FF6E
:10270000204610BDE96300202DE9F04300295FD089
:102710003048314BB3FBF1F381428CBF0A201120CA
:10272000451EB3FBF0F700FB1730ECB220B1022DD1
:102730002846F5D8002037E07D1EB5F5806F33D2EE
:10274000C4EBC40808F103034FEAE30EC3F3C70365
:10275000A4EB030C0EF101094FF47A705FFA8CF6CA
:102760000EFB000E59FA8CFCBEFBFCFCBCF5617F35
:102770001CDC1FFA8CF4581C56FA80F047431648AC
:10278000B0FBF7F7B942D5D1013BDBB20F2BD1D863
:10279000711EC9B207294FF0000005D810711480CE
:1027A0005580537191710120BDE8F08308F1FF332A
:1027B0004FEAE30CC3F3C703E41A0CF1010EE6B2CF
:1027C0000CFB00005EFA84F4B0FBF4F4A4B2D2E790
:1027D0000846E9E73F420F000024F40038B500F551
:1027E0008053114A93F85834D55C4FF454725543D2
:1027F00005F1804303F52443044600211846FFF702
:1028000053F90A4B60612B44A361094B2B44E361EC
:10281000084B2B442362084B2B446362E36A00227B
:10282000C3F8C02038BD00BF1057000870A4004096
:10283000B0A4004088A5004078A600402DE9F04FE4
:1028400000F58055994695F85834022B89B0044616
:102850008A46904604D90027384609B0BDE8F08F73
:10286000994A52F8231009B942F823009749C4F84D
:102870000CA00B7884F8109093B9FFF73DFD944BB2
:102880009A6D42F000729A659A6B42F000729A63F8
:102890009A6B22F000729A6301230B70FFF732FDEE
:1028A00095F85134BBB9FFF727FD8A4A95F858349B
:1028B000D35C012B26D0022B2BD03BB90321152052
:1028C00001F056FD0321162001F052FD012385F889
:1028D0005134FFF717FDFFF70FFDE26A936923F00C
:1028E0001003936100F0E0FB0746E36A9E6916F06F
:1028F000080615D000F0D8FBC31BFA2BF5D9FFF75B
:1029000001FDA8E70321562001F032FD03215720E5
:10291000DAE70321582001F02BFD03215920D3E7EA
:102920009A6942F001029A6100F0BEFB0746E36A31
:102930009A69D00705D400F0B7FBC31BFA2BF6D970
:10294000DDE79A6942F002029A61E36A00275F6557
:10295000FFF7D8FC686CFFF79FFB04F5825B0BF177
:10296000100B202200216846FFF79EF802A8FFF70F
:1029700005FE06976A460BEB06030DF1180E94460A
:10298000BCE80300F44518605960624603F108038F
:10299000F5D1DCF80000186020369CF804201A718C
:1029A000B6F5806FDDD1002304F5A25285F85034CE
:1029B00085F853341A3251462046FFF7A5FE0746E4
:1029C00090B9E26A936923F00103936100F06CFB14
:1029D0000546E36A9B69D9077FF53DAF00F064FBCC
:1029E000431BFA2BF5D936E795F85F6495F85E241A
:1029F000C5F86CA4360246EA426695F86024E36A9C
:102A00001643B5F85C2446EA0246DE61B8F1000FD1
:102A100029D004F5A352023241462046FFF774FE46
:102A200090B9E26A936923F00103936100F03CFBE3
:102A30000546E36A9B69DA077FF50DAF00F034FBCA
:102A4000431BFA2BF5D906E795F8683495F8671417
:102A5000C5F870841B0143EA0123B5F86414E26AE7
:102A600043EA0143D3602046FFF7B8FE002385F810
:102A70005934E36A6FF040421A65E36A164A5A65B0
:102A8000E36A44229A65E36A0722C3F8DC20E36A1A
:102A900003229145DA653FF4DFAEE26A936923F0E1
:102AA0000103936100F000FB0646E36A9B69DB07C4
:102AB00005D500F0F9FA831BFA2BF6D9CBE60123F2
:102AC00085F85234C8E600BFE0630020E8630020C8
:102AD00000100240105700089B0008002DE9F04F3D
:102AE000054689B090469946002741F2680A00F5EC
:102AF0008056EB6AD3F8D430FB40D8074AD505EBB3
:102B0000471252444FEA471B1379190742D4D6F8AB
:102B100080340133C6F8803413799A0648BFD6F85A
:102B2000A83405EB0B0248BF0133524448BFC6F836
:102B3000A834137943F008031371DB0722D596F804
:102B40005334FBB105F58254183468465C44FFF7F2
:102B50001BFD03AB04F1080C206861681A4603C230
:102B6000083464451346F7D120681060A2889A8023
:102B70000123ADF808302B68CDE90089DB6B69468D
:102B800028469847D6F8543423B1D6F89C340133FC
:102B9000C6F89C340137202FABD109B0BDE8F08FC7
:102BA0002DE9F04F8DB004460F4600F07FFA8246C3
:102BB0008946002F56D1E36AD3F89020920141BF95
:102BC00004F58051D1F894240132C1F89424D3F84B
:102BD0009020160703D100200DB0BDE8F08FD3F888
:102BE0009050E669C5F30125482303FB0566E846D6
:102BF0004046FFF7C3FC326851004ABF22F06043F1
:102C0000C2F38A4343F00043920048BF43F080433D
:102C10000093736813F400131FBF04F5805201235F
:102C20008DF80D30D2F8AC340EBF8DF80D30013375
:102C3000C2F8AC34F38803F00F038DF80C304FF07A
:102C4000000B9DF80C0000F08BFA5FFA8BF39842B2
:102C500020D9F2180CA90B44127A03F82C2C0BF192
:102C6000010BEEE7012FB6D1E36AD3F89820950166
:102C700041BF04F58051D1F894240132C1F8942465
:102C8000D3F898201007A6D0D3F89850266AC5F339
:102C90000125A9E7EFB9E36AC3F8945004A8FFF748
:102CA00073FC98E80F0007AD07C52B800023ADF833
:102CB000183023682046CDE904A9DB6B04A99847A6
:102CC00004F5805458B1D4F88C340133C4F88C34F2
:102CD00082E7012F04BFE36AC3F89C50DEE7D4F813
:102CE00090340133C4F89034012075E7F8B50546F7
:102CF0000F4600F58054012639462846FFF750FF5D
:102D000010B184F85364F7E7D4F8543423B1D4F8FD
:102D10009C340133C4F89C34F8BD0000F0B5C36A9C
:102D20001A6C12F47F0F2BD000F580541B6CC4F882
:102D3000A03441F26805002347194FF0010C00EB65
:102D400043122A445E01117911F0020F15D0490790
:102D500013D4B959C66AD6F8C8E00CFA01F111EAE1
:102D60000E0F0AD0C6F8D010117941F0040111718C
:102D7000D4F888240132C4F888240133202BDED112
:102D8000F0BD00002B4B70B51E561B5C012B2FD8DD
:102D9000294D2A4A55F8233052F826400BB341B347
:102DA000236D1A060FD58023236500F07FF950EAC2
:102DB00001020B4602D0013861F10003024655F8CA
:102DC0002600FFF78BFE236D1B032CD555F826300C
:102DD0004FF4002203F580532265012283F8592421
:102DE00021E001232365082323654FF480632365D5
:102DF00070BD236DDA0702D4236D9B0706D503232C
:102E000055F8260023650021FFF770FF236D180792
:102E100002D4236DD90606D5182355F8260023655C
:102E20000121FFF763FF55F82600BDE87040FFF76A
:102E300075BF00BF14570008E06300201857000852
:102E400008B5FFF759FAFFF769FFBDE80840FFF73B
:102E500059BA0000C36AD3F8C40080F40010C0F36C
:102E60004050704700F5805008B5FFF745FA406CB8
:102E7000FFF724F9FFF746FA43090CBF01200020B1
:102E800008BD000000F5805393F8592462B1C16A6F
:102E90008A6922F001028A61D3F898240132C3F8CA
:102EA0009824002283F85924704700002DE9F74345
:102EB00000F5825198461031FFF71EFA002541F2C5
:102EC000680E4FF0010900F5805C00EB4514744476
:102ED00023795E071CD4DB061AD5C36A8E69D3F842
:102EE000C87009FA06F63E4212D04F6801970F6883
:102EF0009742019F77EB08070AD2C3F8D060237985
:102F000043F004032371DCF884340133CCF88434B7
:102F10000135202D01F12001D7D103B0BDE8F043E8
:102F2000FFF7F0B9F8B51E46002313700F460546AB
:102F30001446FFF797FF80F0010038701EB1284655
:102F4000FFF788FF2070F8BD2DE9F04F85B0994656
:102F5000DDE90EA30D4602931378019391F800B0BA
:102F60008046164600F0A2F82B7804460F4613B9A7
:102F70003378002B42D022463B464046FFF796FF6F
:102F8000FFF75EFFFFF77EFF4B4632462946FFF70D
:102F9000C9FF2B7833B1BBF1000F03D0012005B07E
:102FA000BDE8F08F337813B1019B002BF6D108F503
:102FB00080530393029B544577EB03031ED2039B7C
:102FC000D3F85404D0B10368AAEB0401DB6889B2DA
:102FD00098474B46324629464046FFF7A3FF2B78D9
:102FE00013B1BBF1000FD9D1337813B1019B002B82
:102FF000D4D100F05BF804460F46DBE70020CEE7B3
:1030000008B500210846FFF7BDFEBDE8084001F005
:1030100067B8000008B501210020FFF7B3FEBDE846
:10302000084001F05DB8000008B500210120FFF75D
:10303000A9FEBDE8084001F053B8000008B5012121
:103040000846FFF79FFEBDE8084001F049B80000C0
:1030500000B59BB0EFF3098168226846FEF712FDC8
:10306000EFF30583014B9B6BFEE700BF00ED00E033
:1030700008B5FFF7EDFF000000B59BB0EFF3098145
:1030800068226846FEF7FEFCEFF30583014B5B6B9D
:10309000FEE700BF00ED00E0FEE700000FB408B55A
:1030A000029801F0EBFBFEE701F0FCBE01F0D4BE9C
:1030B00013B56C4684E80600031D94E8030083E81A
:1030C0000500012002B010BD73B58568019155B1AE
:1030D0001B885B0707D4D0E900369B6B9847019AA1
:1030E000C1B23046A847012002B070BDF0B5866875
:1030F00089B005460C465EB1BDF838305B070AD48E
:10310000D0E900379B6B98472246C1B23846B0479A
:10311000012009B0F0BD00220023CDE900230023E7
:10312000ADF808300A4603AB01F108061068516893
:103130001C4603C40832B2422346F7D1106820600F
:103140009288A280FFF7B2FF0423ADF808302B6805
:10315000CDE90001DB6B694628469847D8E70000B7
:10316000082817D909280CD00A280CD00B280CD015
:103170000C280CD00D280CD00E2814BF4020302075
:1031800070470C207047102070471420704718209B
:1031900070472020704700002DE9F041456A15B9BD
:1031A0004162BDE8F0814B6823F06047C3F38A4673
:1031B0004FEAD37EC3F3807816EA230638BF3E4633
:1031C000AC462B465A68BEEBD27F22F060440AD050
:1031D000002A18DAA40CB44217D19D420FD10D6019
:1031E000DEE71346EEE7A74207D102F08044C2F3C0
:1031F000807242450BD054B1EFE708D2EDE7CCF82E
:1032000000100B60CDE7B44201D0B442E5D81A6893
:103210009C46002AE5D11960C3E700002DE9F0477C
:10322000089D01F007044FEAD508224405F0070580
:1032300000EBD1004FF47F49944201D1BDE8F08703
:1032400004F0070705F0070A57453E4638BF5646C3
:10325000C6F10806111B8E4228BF0E46E10808EB96
:10326000D50E415C13F80EC0B94029FA06F721FAD1
:103270000AF1FFB28CEA010147FA0AF739408CEAF9
:10328000010C03F80EC034443544D5E780EA012030
:10329000082341F2210201B24000002980B203F16B
:1032A000FF33B8BF504013F0FF03F4D17047000064
:1032B00038B50C468D18A54200D138BD14F8011B55
:1032C000FFF7E4FFF7E7000042684AB11368436084
:1032D0004389818901339BB29942438138BF8381FD
:1032E0001046704770B588B0202204460D466846E7
:1032F0000021FEF7D9FB20460495FFF7E5FF0246C3
:1033000058B16B46054608AE1C4603CCB442286053
:103310006960234605F10805F6D1104608B070BD76
:10332000082817D909280CD00A280CD00B280CD053
:103330000C280CD00D280CD00E2814BF40203020B3
:1033400070470C20704710207047142070471820D9
:103350007047202070470000082817D90C280CD986
:1033600010280CD914280CD918280CD920280CD9CD
:1033700030288CBF0F200E207047092070470A208C
:1033800070470B2070470C2070470D2070470000DD
:103390002DE9F843078C072F04461ED9D0E902987F
:1033A00000254FF6FF73C5F12006A5F1200029FA8C
:1033B00005F108FA06F628FA00F031430143C9B2D4
:1033C0001846FFF763FF0835402D0346EBD1E1694E
:1033D0003A46BDE8F843FFF76BBF4FF6FF70BDE814
:1033E000F883000010B54B6823B9CA8A63F3090259
:1033F000CA8210BD04691A681C600361C38A013B5C
:10340000C3824A60EFE700002DE9F84F1D46CB8AE2
:103410000F46C3F309010529814692460B4630D079
:103420000020AAB207F11A049EB2042E1FFA80F8F7
:103430000FD8904503F1010306D3FB8A0A4462F3D7
:103440000903FB8201201AE01AF80060E6540130FB
:10345000EAE79045F1D2A1F1050B1C237C68BBFB88
:10346000F3F203FB12BB1FFA8BF6002C45D1484642
:10347000FFF72AFF044638B978606FF00200BDE814
:10348000F88F4FF00008E6E7002606607860ADB2DE
:103490004FF0000B454510D90AEB0803221D13F825
:1034A000011B9155B1B208F101081B291FFA88F8D8
:1034B0002BD0454506F10106F1D8FB8AC3F309027A
:1034C000154465F30903BCE7013292B21C46236838
:1034D000002BF9D16B1F0B441C21B3FBF1F301331B
:1034E0009BB29A42D3D2BBF1000FD0D14846FFF72E
:1034F000EBFE20B9C4F800B0BFE70122E7E7C0F84F
:1035000000B05E4620600446C1E74545D5D948462F
:10351000FFF7DAFE08B92060AFE7C0F800B0002678
:1035200020600446B6E700002DE9F04F2DED028B38
:103530001C4683B05B69019207468846002B00F069
:103540009A80238C2BB1E269002A00F09480072B2B
:1035500035D807F10C00FFF7B7FE054638B96FF014
:103560000205284603B0BDEC028BBDE8F08F1422A3
:103570000021FEF799FA228CE16905F10800FEF7B7
:1035800081FA208C013080B2FFF7E6FEFFF7C8FE1B
:10359000013880B22084013028746369228C1B7842
:1035A0002A4403F01F0363F03F0348F00041137205
:1035B000384669602946FFF7EFFD0125D1E700F1A4
:1035C0000C034FF0000908EE103A4FF0800A4E4607
:1035D0004D4618EE100AFFF777FE83460028BED04E
:1035E00014220021FEF760FA002E3AD1019BABF8BD
:1035F000083002220BF1080E1FFA82FC0CF10100C8
:10360000BCF1060F218C80B201D88E422BD3FFF77C
:10361000A3FEFFF785FE62691278013802F01F02EF
:103620008E4208BF4FF0400A42EA49121BFA80F16D
:103630004AEA020A013048F0004281F808A08BF8FB
:103640001000CBF8042059463846FFF7A5FD238C1F
:103650000135B3422DB289F001094FF0000AB8D10B
:103660007FE70022C6E7E169895D0EF802100136A6
:10367000B6B20132C0E76FF0010572E7F8B5154642
:103680000E463022002104461F46FEF70DFA069B27
:103690006360B5F5001F079BA76034BF6A094FF64A
:1036A000FF72A36297B2E66104F1100000239A4210
:1036B00006D800230360A782E3822383E360F8BD7A
:1036C0000660013330462036F1E7000003781BB96D
:1036D0004BB2002BC8BF01707047000000787047E4
:1036E000F8B50C46C969074611B9238C002B37D1B0
:1036F000257E1F2D34D8387828BB228C072A2CD859
:10370000268A36F003032BD14FF6FF70FFF7D0FD6A
:1037100020F001003102400441EA0561400C41EA19
:1037200040254FF6FF72234629463846FFF7FCFE38
:10373000002807DD626913780133DBB21F2B88BFD5
:1037400000231370F8BD218A2D0645EA01250543A3
:103750002046FFF71DFE0246E5E76FF00300F1E7A4
:103760006FF00100EEE7000070B58AB0044616461F
:103770000021282268461D46FEF796F9BDF838302C
:10378000ADF810300F9B05939DF840308DF8183040
:10379000119B07936946BDF84830ADF820302046AC
:1037A000CDE90265FFF79CFF0AB070BD2DE9F0413D
:1037B000D36905460C4616460BB9138C5BBB377EA6
:1037C0001F2F28D895F80080B8F1000F26D030467A
:1037D000FFF7DEFD3378210241EAC33141EA0801F7
:1037E000338A41EA076141EA03410246334641F028
:1037F00080012846FFF798FE00280ADD3378012B68
:1038000007D1726913780133DBB21F2B88BF002305
:103810001370BDE8F0816FF00100FAE76FF003006C
:10382000F7E70000F0B58BB004460D4617460021BF
:10383000282268461E46FEF737F99DF84C305A1E7E
:10384000534253418DF800309DF84030ADF81030B0
:10385000119B05939DF848308DF81830149B079301
:103860006A46BDF85430ADF8203029462046CDE9EF
:103870000276FFF79BFF0BB0F0BD0000406A00B17D
:1038800004307047436A1A68426202691A60036131
:10389000C38A013BC38270472DE9F041D0F82080F4
:1038A000194E14461D464146002709B9BDE8F0816E
:1038B000D1E90223A21A65EB0303964277EB0303D7
:1038C0001ED2036A8B420DD1FFF78CFD036A1B6881
:1038D000036203690B60C38A0161016A013BC38211
:1038E0008846E2E7FFF77EFD0B68C8F80030036901
:1038F0000B60C38A0161013BC382D8F80010D4E792
:1039000088460968D1E700BF80841E002DE9F04F8A
:103910008BB00D46DDF8509014469B46804600283B
:1039200000F01981B9F1000F00F01581531E3F2BF3
:1039300000F21181012A03D1BBF1000F40F00B818D
:103940000023CDE90833B8F81430B5EBC30F4FEAC4
:10395000C30703D300200BB0BDE8F08F2B199F42A3
:10396000D8F80C303ABF7F1BFFB227461BB9D8F8F6
:103970001030002B7AD0272D4ED8C5F12806B7423B
:103980004FF000032CBFF6B23E4600932946D8F80C
:10399000080008AB3246FFF741FCA7EB060A3544A6
:1039A0005FFA8AFAB8F8143003F10053053BDB00E4
:1039B0000493D8F80C3003932821039B13B1BAF178
:1039C000000F2CD1D8F8100040B1BAF1000F05D08B
:1039D000009608AB5246691AFFF720FC38B2002F58
:1039E000B8D066070AD00AAB03EBD401624211F8E3
:1039F000083C02F00702134101F8083C082C3CD9AE
:103A0000102C40F2B580202C40F2B780BBF1000FA3
:103A100000F09C80082334E0BA460026C2E7049BED
:103A2000E02B28BFE02306930B44AB42059314D947
:103A30005A1B03980096924534BF5246D2B2691A77
:103A400008AB04300792FFF7E9FB079A1644AAEB8C
:103A5000020A1544F6B25FFA8AFA049B069A05999F
:103A60009B1A0493039B1B680393A6E70093D8F863
:103A7000080008AB3A462946AEE7BBF1000F13D069
:103A80000123B4EBC30F6CD0082C12D89DF8203062
:103A9000621E23FA02F2D50706D54FF0FF3202FA72
:103AA00004F423438DF820309DF8203089F800304D
:103AB00051E7102C12D8BDF82030621E23FA02F212
:103AC000D10706D54FF0FF3202FA04F42343ADF8D4
:103AD0002030BDF82030A9F800303CE7202C0FD86A
:103AE0000899631E21FA03F3DA0705D54FF0FF3278
:103AF00002FA04F40C430894089BC9F800302AE742
:103B0000402C2BD0DDE90865611EC4F12102A4F12F
:103B1000210326FA01F105FA02F225FA03F3114313
:103B20001943CB0712D50122A4F12003C4F12001CF
:103B300002FA03F322FA01F1A240524243EA0103DE
:103B400063EB430332432B43CDE90823DDE908232C
:103B5000C9E90023FFE66FF00100FCE66FF0080002
:103B6000F9E6082CA0D9102CB3D9202CEED8C3E745
:103B7000BBF1000FADD0022383E7BBF1000FBBD038
:103B800004237EE730B5012A144638BF0124402CB7
:103B900085B028BF40240025012ACDE9025518D858
:103BA0001B788DF8083063070AD004AB03EBD4050B
:103BB000624215F8083C02F00702934005F8083C01
:103BC000009103462246002102A8FFF727FB05B01B
:103BD00030BD082AE4D9102A03D81B88ADF8083074
:103BE000E1E7202A8DBFD3E900231B680293CDE9CA
:103BF0000223D8E710B5CB681BB98B600B618B82B1
:103C000010BD04691A681C600361C38A013BC3824A
:103C1000CA60F0E703064CBFC0F3C0300220704713
:103C200008B50246FFF7F6FF022806D15306C2F395
:103C30000F2001D100F0030008BDC2F30740FBE7ED
:103C40002DE9F04F93B0CDE903230A6804461046EE
:103C5000FFF7E0FF022814BFC2F306260026002A61
:103C60000D46824680F2F28112F0C04940F0EE81AA
:103C7000097B002900F0EA81022803D02378B342AF
:103C800040F0E781C2F304630693104602F07F031D
:103C90000593FFF7C5FF059B29444FEA834848EA8F
:103CA0000A4848EA4668CE7800230022CDE9082376
:103CB000F309834648EA0008029367D0059B009306
:103CC00002466768534608A92046B847002800F016
:103CD000C381276A4FB9414604F10C00FFF702FB8C
:103CE000074690B96FF0020054E03B6998450DD04B
:103CF0003F68002FF9D1414604F10C00FFF7F2FABA
:103D000007460028EED0236A3B60276297F817C069
:103D100006F01F08CCF3840CACEB08001FFA80FE01
:103D20000028B8BF0EF12000A8EB0C031FFA83FE99
:103D3000D7E90221B8BF00B2002B0793BEBF0EF136
:103D400020031BB2079352EA010338D0039BDFF82C
:103D500024E39A1A049B4FF0000C63EB0101964593
:103D60007CEB01032BD36B7B97F81AE0734519D1D9
:103D7000029B002B78D0012821DC7868F8B9DFF8A5
:103D8000F0C2944570EB010316D337E0276A27B9D8
:103D90006FF00C0013B0BDE8F08F3B699845B5D0CB
:103DA0003F68F4E7B24890427CEB010301D3002066
:103DB000F0E7029B002BFAD0079B0F2B17DCFA7D54
:103DC000B30002F0030203F07C031343FB75394692
:103DD0002046FFF707FB6B7BBB76029B3BB9FB7D65
:103DE000C3F38402013262F38603FB75D0E76A7B7A
:103DF000BB7E9A42DBD1029B002B35D0B309022B4C
:103E000032D0039BBB60049BFB60142200210DA8F1
:103E1000FDF74AFE039B0A93049B0B932B1D0C9307
:103E20002B7BADF83EB0013BDBB2ADF83C30069BDE
:103E30008DF84230059B8DF8433094F82C308DF886
:103E400040A083F001038DF844308DF84180A368D1
:103E50000AA920469847FB7DC3F38403013303F08E
:103E60001F039B02FB82A2E7FB7DC6F34012B2EB6D
:103E7000D31F40F0F480C3F38403434540F0F28045
:103E8000029A2B7BB609002A4DD0F2075DD4032B92
:103E900040F2EB80039BBB60049BFB602B7BAE1D61
:103EA000033BDBB23246394604F10C00FFF7ACFAB3
:103EB00000280CDA39462046FFF794FAFB7DC3F35D
:103EC0008403013303F01F039B02FB820AE7DDE951
:103ED0000884AB883B834FF6FF73C9F12000A9F13A
:103EE000200228FA09F104FA00F0014324FA02F250
:103EF00011431846C9B2FFF7C9F909F10809B9F128
:103F0000400F0346E9D1B8822A7B033AD2B2314648
:103F1000FFF7CEF9FB7DB882DA43C2F3C01262F339
:103F2000C713FB7543E786B92E1D013BDBB2324652
:103F3000394604F10C00FFF767FA0028BADB2A7B48
:103F4000B88A013AD2B23146E2E7F98AC1F30901EF
:103F5000013B0429DAB25BD8281D002307F11B06B8
:103F60009A4208D910F801CB06F801C0013101339B
:103F70000529DBB2F4D103990A9104990B9193427C
:103F800007F11B010C9138BF043379680D9134BFE0
:103F900055FA83F300230E93FB8AADF83EB0C3F3CA
:103FA00009031A44069B8DF84230059B8DF8433077
:103FB00094F82C30ADF83C2083F001038DF84430A8
:103FC00000238DF840A08DF841807B602A7BB88A61
:103FD000013A291DFFF76CF93B8BB882834203D16C
:103FE000A3680AA92046984720460AA9FFF702FEBF
:103FF000FB7DBA8AC3F38403013303F01F039B02E2
:10400000FB823B8B9A420CBF00206FF01000C1E690
:104010007B68002BAFD0052001E01C3033461E68C2
:10402000002EFAD1091A081D2E1D184401EB090CA7
:10403000BCF11B0F5FFA89F39DD89A429BD916F801
:10404000013B00F8013B09F10109EFE76FF00900BE
:10405000A0E66FF00A009DE66FF00B009AE66FF0A5
:104060000D0097E66FF00E0094E66FF00F0091E6FA
:1040700040420F0080841E00EFF3098305494A6B1C
:1040800022F001024A63683383F30988002383F333
:104090001188704700EF00E0302080F3118862B68D
:1040A0000C4B0D4AD96821F4E0610904090C0A435C
:1040B000DA60D3F8FC20094942F08072C3F8FC2092
:1040C0000A6842F001020A602022DA7783F82200AF
:1040D000704700BF00ED00E00003FA05001000E0AB
:1040E00010B5302383F311880E4B5B6813F4006323
:1040F00014D0F1EE103AEFF30984683C4FF080736E
:10410000E361094BDB6B236684F3098800F074FBE1
:1041100010B1064BA36110BD054BFBE783F311887B
:10412000F9E700BF00ED00E000EF00E04306000803
:1041300046060008026843681143016003B118474E
:1041400070470000024A136843F0C00313607047D1
:104150000044004013B50E4C204600F0B3FA04F1C1
:1041600014000C49009400234FF4807200F070F9A1
:10417000094B0A4900944FF4807204F1380000F0B2
:10418000E9F9074A074BC4E9172302B010BD00BF85
:10419000F06300205C640020454100085C6500205D
:1041A00000440040007A030A30B5037C214C00290A
:1041B00018BF0C46012B0CD11F4B984209D11F4B45
:1041C0009A6D42F400329A659A6F42F400329A670F
:1041D0009B6F2268036EC16D846603EB5203B3FBD1
:1041E000F2F36268150442BF23F0070503F00703EA
:1041F00043EA4503CB60A36843F040034B60E368A8
:1042000043F001038B6042F4967343F001030B60AB
:104210004FF0FF330B62510505D512F0102205D087
:10422000B2F1805F04D080F8643030BD7F23FAE7BC
:104230003F23F8E768570008F063002000100240B1
:104240002DE9F047C66D3768F469346221070546E9
:1042500019D014F0080118BF4FF48071E20748BF6D
:1042600041F02001A30748BF41F04001600748BF6B
:1042700041F08001302383F31188281DFFF75AFF96
:10428000002383F31188E2050AD5302383F31188D4
:104290004FF48061281DFFF74DFF002383F3118841
:1042A0004FF030094FF0000A14F0200838D13B06D7
:1042B00016D54FF0300905F1380A200610D589F3DC
:1042C0001188504600F07AF9002836DA0821281DB6
:1042D000FFF730FF27F080033360002383F311885A
:1042E000790614D5620612D5302383F31188D5E9F7
:1042F00013239A4208D12B6C33B11021281D27F0CB
:104300004007FFF717FF3760002383F31188E306A8
:1043100018D5AA6E1369ABB1BDE8F04750691847CC
:1043200089F31188736A95F864102846194000F0E3
:10433000E3F98AF31188F469B6E7B06288F311886B
:10434000F469BAE7BDE8F0874FF0E023002258682F
:104350004FF0FF31930003F1604303F561430132F5
:104360009042C3F88010C3F88011F3D27047000068
:1043700000F1604303F561430901C9B283F80013FA
:10438000012200F01F039A4043099B0003F16043A0
:1043900003F56143C3F880211A607047F8B51546EC
:1043A00082680669AA420B46816938BF8568761A19
:1043B000B54204460BD218462A46FDF763FBA369B3
:1043C0002B44A361A3685B1BA3602846F8BD0CD9EE
:1043D00018463246FDF756FBAF1BE1683A463044BB
:1043E000FDF750FBE3683B44EBE718462A46FDF730
:1043F00049FBE368E5E7000083689342F7B515469B
:10440000044638BF8568D0E90460361AB5420BD23D
:104410002A46FDF737FB63692B446361A36828468E
:104420005B1BA36003B0F0BD0DD932460191FDF7CF
:1044300029FB0199E068AF1B3A463144FDF722FBA6
:10444000E3683B44E9E72A46FDF71CFBE368E4E741
:1044500010B50A440024C361029B8460C0E90000D7
:10446000C0E90511C1600261036210BD08B5D0E961
:104470000532934201D1826882B98268013282603A
:104480005A1C42611970D0E904329A4224BFC368B1
:104490004361002100F078FA002008BD4FF0FF30A2
:1044A000FBE7000070B5302304460E4683F3118805
:1044B000A568A5B1A368A269013BA360531CA361D1
:1044C00015782269934224BFE368A361E3690BB1C5
:1044D00020469847002383F31188284607E0314699
:1044E000204600F041FA0028E2DA85F3118870BD19
:1044F0002DE9F74F04460E4617469846D0F81C9013
:104500004FF0300A8AF311884FF0000B154665B161
:104510002A4631462046FFF741FF034660B941462F
:10452000204600F021FA0028F1D0002383F31188FF
:10453000781B03B0BDE8F08FB9F1000F03D00190F4
:104540002046C847019B8BF31188ED1A1E448AF35D
:104550001188DCE7C0E90511C160C3611144009B0B
:104560008260C0E90000016103627047F8B504464B
:104570000D461646302383F31188A768A7B1A368B8
:10458000013BA36063695A1C62611D70D4E9043267
:104590009A4224BFE3686361E3690BB12046984700
:1045A000002080F3118807E03146204600F0DCF956
:1045B0000028E2DA87F31188F8BD0000D0E905236E
:1045C0009A4210B501D182687AB98268013282605C
:1045D0005A1C82611C7803699A4224BFC3688361B4
:1045E000002100F0D1F9204610BD4FF0FF30FBE76D
:1045F0002DE9F74F04460E4617469846D0F81C9012
:104600004FF0300A8AF311884FF0000B154665B160
:104610002A4631462046FFF7EFFE034660B9414681
:10462000204600F0A1F90028F1D0002383F311887F
:10463000781B03B0BDE8F08FB9F1000F03D00190F3
:104640002046C847019B8BF31188ED1A1E448AF35C
:104650001188DCE7026843681143016003B1184721
:10466000704700001430FFF743BF00004FF0FF33E6
:104670001430FFF73DBF00003830FFF7B9BF00002E
:104680004FF0FF333830FFF7B3BF00001430FFF7AF
:1046900009BF00004FF0FF311430FFF703BF0000E7
:1046A0003830FFF763BF00004FF0FF323830FFF7BC
:1046B0005DBF0000012914BF6FF013000020704798
:1046C000FFF748BD044B03600023C0E90233436099
:1046D00001230374704700BF8057000810B53023D2
:1046E000044683F31188FFF75FFD02232374002043
:1046F00080F3118810BD000038B5C36904460D462B
:104700001BB904210844FFF7A5FF294604F1140052
:10471000FFF7ACFE002806DA201D4FF40061BDE86B
:104720003840FFF797BF38BD0023037582680369DF
:104730001B6899689142FBD25A680360426010601E
:104740005860704700230375826803691B68996885
:104750009142FBD85A68036042601060586070470D
:1047600008B50846302383F311880B7D032B05D051
:10477000042B0DD02BB983F3118808BD8B6900225F
:104780001A604FF0FF338361FFF7CEFF0023F2E79B
:10479000D1E9003213605A60F3E70000FFF7C4BFAD
:1047A000054BD9680875186802681A6053600122C1
:1047B0000275D860FBF730BF6066002030B50C4B47
:1047C000DD684B1C87B004460FD02B46094A68466B
:1047D00000F06CF92046FFF7E3FF009B13B1684639
:1047E00000F06EF9A86907B030BDFFF7D9FFF9E70F
:1047F0006066002061470008044B1A68DB68906817
:104800009B68984294BF002001207047606600209A
:10481000084B10B51C68D86822681A6053600122E2
:104820002275DC60FFF78EFF01462046BDE8104090
:10483000FBF7F2BE60660020044B1A68DB689268E2
:104840009B689A4201D9FFF7E3BF7047606600207A
:1048500038B5074C074908480123002523706560D7
:1048600000F01EFC0223237085F3118838BD00BFC1
:10487000C8680020AC5700086066002008B572B612
:10488000044B186500F0D4FA00F08CFB024B0322B5
:104890001A70FEE760660020C868002000F046B984
:1048A000EFF3118020B9EFF30583302282F31188F2
:1048B0007047000010B530B9EFF30584C4F3080465
:1048C00014B180F3118810BDFFF7B6FF84F311888F
:1048D000F9E700008B60022308618B82084670476D
:1048E0008368A3F1840243F8142C026943F8442C32
:1048F000426943F8402C094A43F8242CC26843F823
:10490000182C022203F80C2C002203F80B2C044A6A
:1049100043F8102CA3F12000704700BF31060008B7
:104920006066002008B5FFF7DBFFBDE80840FFF731
:1049300035BF0000024BDB6898610F20FFF730BFE6
:1049400060660020302383F31188FFF7F3BF000077
:1049500008B50146302383F311880820FFF72EFFA6
:10496000002383F3118808BD064BDB6839B1426828
:1049700018605A60136043600420FFF71FBF4FF0B8
:10498000FF307047606600200368984206D01A68BE
:104990000260506099611846FFF700BF7047000041
:1049A00010B503689C68A2420CD85C688A600B60F2
:1049B0004C602160596099688A1A9A604FF0FF3301
:1049C000836010BD1B68121BECE700000A2938BF8A
:1049D0000A2170B504460D460A26601900F05AFBFC
:1049E00000F046FB041BA54203D8751C2E46044666
:1049F000F3E70A2E04D9BDE87040012000F090BB17
:104A000070BD0000F8B5144B0D46D96103F11001DB
:104A100041600A2A1969826038BF0A220160486031
:104A20001861A818144600F027FB0A2700F020FBA5
:104A3000431BA342064606D37C1C281900F02AFB20
:104A400027463546F2E70A2F04D9BDE8F840012091
:104A500000F066BBF8BD00BF60660020F8B50646F2
:104A60000D4600F005FB0F4A134653F8107F9F4296
:104A700006D12A4601463046BDE8F840FFF7C2BFDE
:104A8000D169BB68441A2C1928BF2C46A34202D90D
:104A90002946FFF79BFF224631460348BDE8F84010
:104AA000FFF77EBF606600207066002010B4C0E98A
:104AB000032300235DF8044B4361FFF7CFBF0000E1
:104AC00010B5194C236998420DD0D0E900328168A5
:104AD00013605A609A680A449A60002303604FF09A
:104AE000FF33A36110BD2346026843F8102F5360C3
:104AF0000022026022699A4203D1BDE8104000F012
:104B0000C3BA936881680B44936000F0B1FA2269DC
:104B1000E1699268441AA242E4D91144BDE8104008
:104B2000091AFFF753BF00BF606600202DE9F04768
:104B3000DFF8BC8008F110072C4ED8F8105000F0B8
:104B400097FAD8F81C40AA68031B9A423ED814442E
:104B5000D5E900324FF00009C8F81C4013605A60D4
:104B6000C5F80090D8F81030B34201D100F08CFAAB
:104B700089F31188D5E9033128469847302383F318
:104B800011886B69002BD8D000F072FA6A69A0EB2B
:104B900004094A4582460DD2022000F0C1FA0022E3
:104BA000D8F81030B34208D151462846BDE8F04746
:104BB000FFF728BF121A2244F2E712EB090938BFA7
:104BC0004A4629463846FFF7EBFEB5E7D8F81030DD
:104BD000B34208D01444211AC8F81C00A960BDE8EB
:104BE000F047FFF7F3BEBDE8F08700BF7066002016
:104BF0006066002000207047FEE70000704700005C
:104C00004FF0FF3070470000BFF34F8F024A136927
:104C1000DB03FCD4704700BF0020024008B5094BFD
:104C20001B7873B9FFF7F0FF074B5A69002ABFBF23
:104C3000064A9A6002F188329A601A6822F4806209
:104C40001A6008BDE068002000200240230167458B
:104C500008B50B4B1B7893B9FFF7D6FF094B5A6980
:104C600042F000425A611A6842F480521A601A688F
:104C700022F480521A601A6842F480621A6008BDF9
:104C8000E068002000200240FF289ABF00F5803035
:104C9000C0020020704700004FF400607047000021
:104CA0004FF4807070470000FF2808B50BD8FFF75D
:104CB000EBFF00F500630268013204D10430834247
:104CC000F9D1012008BD0020FCE70000FF2810B545
:104CD00004461FD8FFF798FFFFF7A0FF0E4BF32203
:104CE0001A6102225A615A6942EAC0025A615A693B
:104CF00042F480325A61FFF787FF4FF40061FFF7FB
:104D0000C3FF00F04BF9FFF7A3FF2046BDE81040BA
:104D1000FFF7CABF002010BD002002402DE9F84374
:104D200040EA020313F00703144606D0304B40F26A
:104D300031321A600020BDE8F88385182D4A95426B
:104D40000CD92B4A40F236311160F3E7031D1B6882
:104D50004A68934208D1083C08300831072C14D91E
:104D600002680B689A42F1D0FFF758FFFFF74CFF3B
:104D7000214E08314FF001084FF00009012CA1F13C
:104D8000080706D8FFF764FF01E0002CECD10120F2
:104D9000D1E7C6F81480054651F8083C45F8043BB5
:104DA00051F8043C4360FFF72FFF336943F00103E0
:104DB0003361C6F81490026851F8083C9A420CD04E
:104DC0000B4B40F25E321A600C4B18600C4B1C60AF
:104DD0000C4B1F60FFF73CFFACE72D6851F8043C1B
:104DE0009D4201F10801EBD1083C0830C6E700BF45
:104DF000DC6800200000080800200240D068002085
:104E0000D8680020D4680020084908B50B7828B17C
:104E10001BB9FFF703FF01230B7008BD002BFCD06B
:104E2000BDE808400870FFF713BF00BFE06800202E
:104E300008B54FF4C0314FF0005000F0B1F8BDE8B4
:104E400008404FF400414FF0805000F0A9B8000036
:104E5000084600F0F3BB000070B582B0FFF720FDFC
:104E60000E4E054600F004F93268904237BF0C4AF6
:104E70000B49516814682EBFD1E9004101315160DE
:104E80000419034641F10001284601913360FFF700
:104E900011FD0199204602B070BD00BFE4680020FA
:104EA000E868002070B582B0FFF7FAFC104E0546A6
:104EB00000F0DEF83268904237BF0E4A0D49516863
:104EC00014682EBFD1E9004101315160041941F14C
:104ED00000010346284601913360FFF7EBFC01997E
:104EE0004FF47A7200232046FBF782F902B070BDBE
:104EF000E4680020E86800200244D2B2904200D169
:104F00007047431C800000F1804000F51450006899
:104F100041F8040BD8B2F1E7124B10B5D3F890402A
:104F2000240409D4D3F89040C3F89040D3F89040BB
:104F300044F40044C3F890400B4C2368024443F40B
:104F400080732360D2B2904200D110BD431C800018
:104F500000F1804000F5145051F8044B0460D8B2C1
:104F6000F1E700BF001002400070004007B50122C9
:104F700001A90020FFF7C0FF019803B05DF804FB12
:104F800013B50446FFF7F2FFA04205D0012201A9A4
:104F900000200194FFF7C0FF02B010BD7047000071
:104FA0007047000070470000074B45F255521A60E9
:104FB00002225A6040F6FF729A604CF6CC421A60A8
:104FC000024B01221A70704700300040F468002044
:104FD000034B1B781BB1034B4AF6AA221A60704799
:104FE000F468002000300040054B1A6832B902F125
:104FF000804202F50432D2F894201A60704700BF54
:10500000F0680020024B4FF40002C3F89420704770
:105010000010024008B5FFF7E7FF024B1868C0F325
:10502000407008BDF068002070470000FEE70000F7
:105030000A4B0B480B4A90420BD30B4BDA1C121A4B
:10504000C11E22F003028B4238BF00220021FCF770
:105050002BBD53F8041B40F8041BECE71C59000857
:1050600078690020786900207869002000F0C2B8D3
:105070004FF08043586A70474FF0804300225863D6
:105080001A610222DA6070474FF080430022DA6032
:10509000704700004FF0804358637047FEE7000000
:1050A00070B51B4B01630025044686B058608562CD
:1050B0000E46FEF7F1FF04F11003C4E904334FF08C
:1050C000FF33C4E90635C4E90044A560E562FFF793
:1050D000CFFF2B460246C4E9082304F134010D4AF0
:1050E000256580232046FFF7F5FB0123E0600A4A8F
:1050F0000375009272680192B268CDE90223074BF2
:105100006846CDE90435FFF70DFC06B070BD00BF61
:10511000C8680020B8570008BD5700089D50000817
:10512000024AD36A1843D062704700BF606600200D
:105130004B6843608B688360CB68C3600B694361D5
:105140004B6903628B6943620B6803607047000020
:1051500008B5204BDA6A42F07F02DA62DA6A22F09E
:105160007F02DA62DA6ADA6C42F07F02DA64DA6EBF
:1051700042F07F02DA66184ADB6E11464FF090402B
:10518000FFF7D6FF02F11C0100F58060FFF7D0FFAA
:1051900002F1380100F58060FFF7CAFF02F1540107
:1051A00000F58060FFF7C4FF02F1700100F5806038
:1051B000FFF7BEFF02F18C0100F58060FFF7B8FF3A
:1051C00002F1A80100F58060FFF7B2FFBDE80840DA
:1051D00000F050B800100240C457000808B500F0B5
:1051E000FBF9FFF735FBBDE80840FFF7FDBE000007
:1051F000704700000F4B9A6D42F001029A659A6F5A
:1052000042F001029A670C4A9B6F936843F00103D6
:1052100093604FF08043A7229A624FF0FF32DA6228
:1052200000229A615A63DA605A6001225A611A6058
:10523000704700BF00100240002004E04FF08042A1
:1052400008B51169D3680B40D9B2C9439B071161F6
:1052500007D5302383F31188FFF720FB002383F366
:10526000118808BD08B5FFF76FF8BDE8084000F0E9
:105270008BB900004E4B4FF0FF319A6A99629A6ADF
:1052800000229A62986AD86A60F07F00D862D86A71
:1052900000F07F00D862D86A186B1963186B1A6324
:1052A000186B986B9963986B9A63986BD86BD963FA
:1052B000D86BDA63D86B186C1964196C1A64196CA2
:1052C000196E41F001011966D3F8801021F0010137
:1052D000C3F88010D3F88010996D41F08051996522
:1052E000996F21F080519967996F32494FF40040CE
:1052F0008860CA600A624A628A62CA620A634A6352
:105300008A63CA630A644A648A64CA640A654A652D
:105310004A604FF48072C1F880204FF440720A60F6
:105320004A6912F48062FBD1D3F8901011F4407FE7
:105330001EBF4FF48031C3F89010C3F89020D3F80B
:10534000982042F00102C3F89820D3F898209207E1
:10535000FBD51A6842F480321A601A689003FCD5B3
:10536000D3F8902022F00322C3F89020124ADA608A
:105370001A6842F080721A601A689101FCD50F49D0
:105380000F4800229A60C3F888100E49C3F89C2089
:10539000016002684A401207FBD19A6842F003029A
:1053A0009A609A6802F00C020C2AFAD1704700BF8A
:1053B0000010024000700040132A610155010050A6
:1053C0000020024004070400074A08B5536903F0AF
:1053D0000103536123B1054A13680BB15068984724
:1053E000BDE80840FEF77CBE00040140F8680020DC
:1053F000074A08B5536903F00203536123B1054A14
:1054000093680BB1D0689847BDE80840FEF768BEC6
:1054100000040140F8680020074A08B5536903F00A
:105420000403536123B1054A13690BB150699847CE
:10543000BDE80840FEF754BE00040140F8680020B3
:10544000074A08B5536903F00803536123B1054ABD
:1054500093690BB1D0699847BDE80840FEF740BE9C
:1054600000040140F8680020074A08B5536903F0BA
:105470001003536123B1054A136A0BB1506A984770
:10548000BDE80840FEF72CBE00040140F86800208B
:10549000164B10B55C6904F478725A61A30604D502
:1054A000134A936A0BB1D06A9847600604D5104A34
:1054B000136B0BB1506B9847210604D50C4A936BC4
:1054C0000BB1D06B9847E20504D5094A136C0BB1B8
:1054D000506C9847A30504D5054A936C0BB1D06C6A
:1054E0009847BDE81040FEF7FBBD00BF0004014037
:1054F000F8680020194B10B55C6904F47C425A61CD
:10550000620504D5164A136D0BB1506D98472305FB
:1055100004D5134A936D0BB1D06D9847E00404D5C0
:105520000F4A136E0BB1506E9847A10404D50C4A74
:10553000936E0BB1D06E9847620404D5084A136F7E
:105540000BB1506F9847230404D5054A936F0BB1F4
:10555000D06F9847BDE81040FEF7C2BD000401407F
:10556000F868002008B50348FEF76AFEBDE8084069
:10557000FEF7B6BDF063002008B5FFF75FFEBDE89B
:105580000840FEF7ADBD0000062108B50846FEF74D
:10559000EFFE06210720FEF7EBFE06210820FEF7AE
:1055A000E7FE06210920FEF7E3FE06210A20FEF7AA
:1055B000DFFE06211720FEF7DBFE06212820FEF77E
:1055C000D7FE07211C20FEF7D3FEBDE808400C21C2
:1055D0002620FEF7CDBE000008B5FFF743FE00F021
:1055E00009F8FFF76DF8FFF703FEBDE80840FFF785
:1055F0003DBD00000023054A19460133102BC2E9C6
:10560000001102F10802F8D1704700BFF8680020CD
:105610000B460146184600F003B8000000F00EB833
:1056200010B5054C13462CB10A4601460220AFF3D3
:10563000008010BD2046FCE700000000024B014640
:105640001868FFF705BC00BF2823002010B50139FA
:105650000244904201D1002005E0037811F8014F87
:10566000A34201D0181B10BD0130F2E72DE9F04133
:10567000A3B1C91A17780144044603F1FF3C8C42D8
:10568000204601D9002009E00578BD4204F101045B
:10569000F5D10CEB0405D618A54201D1BDE8F08187
:1056A00015F8018D16F801EDF045F5D0E7E700009B
:1056B000034611F8012B03F8012B002AF9D170479A
:1056C0006F72672E6172647570696C6F742E486FAB
:1056D0006C7962726F47345F4750530053544D33B7
:1056E0003247343F3F00000040A2E4F16468910675
:1056F0000041A3E5F2656992070000004261642061
:1057000043414E496661636520696E6465782E0089
:10571000000100000001FF0000640040006800403C
:1057200000000000000000003D28000819230008C8
:10573000492F000811230008C1230008A5250008EF
:105740008923000851230008552300082D23000851
:10575000152300086525000839230008B13000082A
:1057600045230008392500080096000000000000CD
:105770000000000000000000000000000000000029
:1057800000000000814600086D460008A946000898
:1057900095460008A14600088D4600087946000895
:1057A00065460008B546000863300000A8570008A9
:1057B000B8660020C86800206D61696E0069646C7D
:1057C00065000000A000802A00000000AAAAAAAA82
:1057D00050000024FFFF0000007700000090090047
:1057E0000400005A00000000AAAAAA9A04000000BF
:1057F000FFBF00000000000000009900001110141D
:1058000000000000AAAAAAA600010010FFDF000005
:105810000000000000000000000000000000000088
:10582000AAAAAAAA00000000FFFF000000000000D2
:10583000000000000000000000000000AAAAAAAAC0
:1058400000000000FFFF000000000000000000005A
:105850000000000000000000AAAAAAAA00000000A0
:10586000FFFF00000000000000000000000000003A
:1058700000000000AAAAAAAA00000000FFFF000082
:10588000000000000000000098A9FF7F0100000058
:105890001D04000000000000007007000000000070
:1058A000FE2A0100D2040000FF000000F063002087
:1058B00000000000DC5600082C230020000000003F
:1058C00000000000000000000000000000000000D8
:1058D00000000000000000000000000000000000C8
:1058E00000000000000000000000000000000000B8
:1058F00000000000000000000000000000000000A8
:105900000000000000000000000000000000000097
:0C5910000000000000000000000000008B
:00000001FF
